:020000040000FA
:02000000912845
:08000800512882070A34063476
:100010000A3406340A340334FA30000000000000C9
:100020000000FF3E031D0D2808000C200C200C20B2
:100030000C20080086001520860164300D20080081
:1000400011081A2010081A200F081A200E081A206A
:1000500008004030950031282030950031281030BC
:10006000950015080605031931280A300D201508DA
:10007000060503193128080000306500703066005D
:1000800000300630043062000030910009309000EA
:1000900005308F0000308E008D008C00A0308B006A
:1000A00008009200030E9300040E94000C308400AC
:1000B000800A0C30040205200002031D672880011D
:1000C000840A911C5828101D582890019101130E84
:1000D0008300140E8400920E120E0B110900800A88
:1000E0000E3004020520000203198001000886007A
:1000F000152008008600061E6F20861A7B282C20FB
:10010000840A08008B130E3084002C2001307A20E2
:1001100002307A2004307A2008307A2086018B174A
:0E01200008003C20061F2020861E8220922808
:02400E00F03F81
:00000001FF
